:020000040000FA
:04000000CB303A289F
:040004000034003490
:08000800A000030EA100831209
:100010008B1C32288B1032181428B21C3228643002
:10002000010203183128182800001628172818285C
:1000300019281A281B281C281D281E281F283210A2
:10004000B214A810031005190314AA0DA90DA80DC8
:10005000B10B322832152A08AF002908AE00280853
:10006000AD00B21081010B11210E8300A00E200EF5
:02007000090085
:0C007400203084008001840A80300402E7
:10008000031C3C281230B100E52183160C30850595
:1000900087018312850187010730990000309A009B
:1000A000103083168E008312603083168F00831207
:1000B00000308316910000008312C830831681003F
:1000C000831231309000003083168C008312103080
:1000D0008B00BD1B7128851971286400851D6D2852
:1000E000FB22E22281018E018F010B118B100B107C
:1000F0008C018B17892032199F20B40B872803109D
:1001000085190314BA0DF0303A0203194521212351
:100110007A286400321808000B1D08000B11B21079
:1001200032141230B100051D9A28331483160113BE
:10013000831208003310831601178312080032114E
:100140000130B7008B132030370783169B001C1437
:100150001A088312A400A500C030A5061030370786
:1001600083169B001C141A088312A3000030370763
:1001700083169B001C141A088312A2008B17331CD1
:10018000C72822090339A200A309A409A509220846
:100190002D02031D3F2923082E02031D3F29240899
:1001A0002F02031D3F2901303702031DDC283E18B2
:1001B000DC283E143F14072202303702031DE528D5
:1001C000BE18E528BE143F14132203303702031D66
:1001D000EE283E19EE283E153F141F220430370248
:1001E000031DF728BE19F728BE153F142B22053032
:1001F0003702031D00293E1A00293E163F143722FC
:1002000006303702031D0929BE1A0929BE163F14FC
:10021000462207303702031D12293E1B12293E17C2
:100220003F14582208303702031D1B29BE1B1B290F
:10023000BE173F14632209303702031D24295E18BC
:1002400024295E143F146E220A303702031D2D2923
:10025000DE182D29DE143F1479220B303702031DDE
:1002600036295E1936295E153F1484220C30370278
:10027000031D3F29DE193F29DE153F149222B70ADC
:100280000D30370203180800A2280130B600B40070
:10029000B500B70085018701B213DF228920B40BB6
:1002A0005E29031085190314BA0DF0303A020319C0
:1002B0008529B50B5E299630B5009121321D4E2956
:1002C0003211331C68292D090339AD00AE09AF097D
:1002D0002F1CB2132F1C4E29B21B4E292E184E294B
:1002E000B2178B1320303707BC002F08BB00D0217A
:1002F00010303707BC002E08BB00D0210030370774
:10030000BC002D08BB00D0218B1785018701B70ADF
:10031000B6010130B5000D303702031C4E29E22230
:100320000800013037020319A322023037020319F3
:10033000A822033037020319AD2204303702031913
:10034000B222053037020319B722063037020319EB
:10035000BC22073037020319C122083037020319C3
:10036000C622093037020319CB220A30370203199B
:10037000D0220B3037020319D5220C303702031973
:10038000DA2208003F1C08003F101030BC003E0875
:10039000BB00D0213030BC005E08BB00D02108007B
:1003A0008B133B0883161C159A0083123C08831696
:1003B0009B0055309D00AA309D009C1464009C1841
:1003C000DE291C1183128B170800831600309B0056
:1003D0001C141A088312BD00831610309B001C14D5
:1003E0001A088312BE00831630309B001C141A08B2
:1003F0008312DE00FF30C800CA15CB15CC15CD1511
:10040000CE15CF15D015D115D215D3150800C13092
:10041000BE05FF30DE050130C405C0000030C2005B
:10042000C6005F100800C230BE05FF30DE05023096
:10043000C405C0000030C200C6005F100800C43010
:10044000BE05FF30DE050630C405C0000030C20026
:10045000C6005F100800C830BE05FF30DE050A3058
:10046000C405C0000030C200C6005F100800D030D4
:10047000BE05FF30DE053D181030BD181130C40533
:10048000C0000030C200C6005F100800E030BE05AA
:10049000FF30DE053D181830BD181930C405C00006
:1004A0001830C200C6005F105F17C4114412080064
:1004B0007F30BE05C030DE050830C505C100003004
:1004C000C300C7000800BF30BE05C030DE051030D5
:1004D000C505C1000030C300C70008003F30BE059D
:1004E000C130DE053030C505C1000030C300C70093
:1004F00008003F30BE05C230DE055030C505C100E2
:100500000030C300C70008003F30BE05C430DE0520
:100510003D188030BD188830C505C1000030C300CB
:10052000C70008003F30BE05C830DE053D18C030AA
:10053000BD18C830C505C100C030C300C700DF17F3
:100540004513C513080010308506003087060800E3
:1005500020308506003087060800213085060030EF
:100560008706080022308506003087060800003024
:1005700085060230870608000230850602308706AD
:100580000800003085060430870608000030850624
:1005900001308706080000308506213087060800F4
:1005A00000308506113087060800003085060830C7
:1005B00087060800003085061830870608003E18B8
:1005C000A32208003E180722BE1813223E191F223C
:1005D000BE192B223E1A3722BE1A46223E1B582233
:1005E000BE1B63225E186E22DE1879225E198422F9
:1005F000DE1992220800B601B401B5013D1C032B9F
:10060000BD01BD14052BBD013D143D08B6006400BD
:10061000092B0A2B0B2B0C2B0D2BFF30B51B850048
:10062000B51F8501B40B072BB50B072B0310B60CB8
:10063000B608031D072B0030BC003D08BB00D021CD
:1006400008008F08031908008F0178308E00C80F4A
:100650004B2DC80A441C512B461C422BCA1C332B61
:10066000CA014A155F2B4A1D382BCA01CA155F2BD8
:10067000CA1D3D2BCA014A165F2B4A1E5F2BCA01B9
:10068000CA145F2B4A1D472BCA014A165F2BCA1D8D
:100690004C2BCA014A165F2B4A1E5F2BCA01CA1493
:1006A0005F2BCA1C562BCA014A155F2B4A1D5B2BB8
:1006B000CA01CA155F2B4A1E5F2BCA014A15C41C0A
:1006C000862BC61C772BCB1C682BCB014B15942B90
:1006D0004B1D6D2BCB01CB15942BCB1D722BCB015E
:1006E0004B16942B4B1E942BCB01CB14942B4B1DF0
:1006F0007C2BCB014B16942BCB1D812BCB014B16A6
:10070000942B4B1E942BCB01CB14942BCB1C8B2BFB
:10071000CB014B15942B4B1D902BCB01CB15942B60
:100720004B1E942BCB014B15441DBB2B461DAC2BF4
:10073000CC1C9D2BCC014C15C92B4C1DA22BCC01E4
:10074000CC15C92BCC1DA72BCC014C16C92B4C1E8C
:10075000C92BCC01CC14C92B4C1DB12BCC014C1690
:10076000C92BCC1DB62BCC014C16C92B4C1EC92B4A
:10077000CC01CC14C92BCC1CC02BCC014C15C92BE3
:100780004C1DC52BCC01CC15C92B4C1EC92BCC0143
:100790004C15C41DF12BC61DE22BCD1CD32BCD0156
:1007A0004D155F13FF2B4D1DD82BCD01CD15FF2B04
:1007B000CD1DDD2BCD014D16FF2B4D1EFF2BCD0189
:1007C000CD14FF2B4D1DE72BCD014D16FF2BCD1D5D
:1007D000EC2BCD014D16FF2B4D1EFF2BCD01CD1463
:1007E000FF2BCD1CF62BCD014D15FF2B4D1DFB2BEB
:1007F000CD01CD15FF2B4D1EFF2BCD014D155F1BE0
:10080000282C441E282C461E192CCE1C0A2CCE0146
:100810004E15362C4E1D0F2CCE01CE15362CCE1D6E
:10082000142CCE014E16362C4E1E362CCE01CE1474
:10083000362C4E1D1E2CCE014E16362CCE1D232CD2
:10084000CE014E16362C4E1E362CCE01CE14362C32
:10085000CE1C2D2CCE014E15362C4E1D322CCE0129
:10086000CE15362C4E1E362CCE014E15C51D5D2CD8
:10087000C71D4E2CCF1C3F2CCF014F156B2C4F1D8D
:10088000442CCF01CF156B2CCF1D492CCF014F1617
:100890006B2C4F1E6B2CCF01CF146B2C4F1D532C88
:1008A000CF014F166B2CCF1D582CCF014F166B2C40
:1008B0004F1E6B2CCF01CF146B2CCF1C622CCF01A1
:1008C0004F156B2C4F1D672CCF01CF156B2C4F1E76
:1008D0006B2CCF014F15451E922C471E832CD01C2C
:1008E000742CD0015015A02C501D792CD001D0159E
:1008F000A02CD01D7E2CD0015016A02C501EA02C58
:10090000D001D014A02C501D882CD0015016A02C42
:10091000D01D8D2CD0015016A02C501EA02CD00123
:10092000D014A02CD01C972CD0015015A02C501DF9
:100930009C2CD001D015A02C501EA02CD0015015FD
:10094000C51EC72CC71EB82CD11CA92CD10151150E
:10095000D52C511DAE2CD101D115D52CD11DB32CC8
:10096000D1015116D52C511ED52CD101D114D52C25
:10097000511DBD2CD1015116D52CD11DC22CD10138
:100980005116D52C511ED52CD101D114D52CD11CEA
:10099000CC2CD1015115D52C511DD12CD101D11503
:1009A000D52C511ED52CD1015115451FFD2C471FAB
:1009B000EE2CD21CDF2CD2015215DF130B2D521D51
:1009C000E42CD201D2150B2DD21DE92CD2015216E6
:1009D0000B2D521E0B2DD201D2140B2D521DF32CB8
:1009E000D20152160B2DD21DF82CD20152160B2D0E
:1009F000521E0B2DD201D2140B2DD21C022DD2016E
:100A000052150B2D521D072DD201D2150B2D521E42
:100A10000B2DD2015215DF1B342DC51F342DC71FDE
:100A2000252DD31C162DD3015315422D531D1B2DDF
:100A3000D301D315422DD31D202DD3015316422DA2
:100A4000531E422DD301D314422D531D2A2DD30101
:100A50005316422DD31D2F2DD3015316422D531E55
:100A6000422DD301D314422DD31C392DD30153155C
:100A7000422D531D3E2DD301D315422D531E422D21
:100A8000D3015315C2214008C4004108C5005F18B6
:100A9000DF145F1CDF104808C9000C304A05031D35
:100AA00005120C304B05031D85120C304C05031D3F
:100AB00005100C304D05031D85100C304E05031D2F
:100AC00087100C304F05031D07110C305005031D16
:100AD00007100C305105031D87120C305205031D01
:100AE00007120C305305031D871149080E02031825
:100AF000A52D12304A05031D051612304B05031DA6
:100B0000851612304C05031D051412304D05031DCA
:100B1000851412304E05031D871412304F05031D36
:100B2000071512305005031D071412305105031D1F
:100B3000871612305205031D071612305305031D88
:100B40008715FF304802031908008F08031D0800AD
:100B5000892049080E02031CA52D18304A05031DE3
:100B6000051206304A05031D051618304B05031DF6
:100B7000851206304B05031D851618304C05031DE4
:100B8000051006304C05031D051418304D05031DD6
:100B9000851006304D05031D851418304E05031DC4
:100BA000871006304E05031D871418304F05031DAE
:100BB000071106304F05031D071518305005031D9A
:100BC000071006305005031D071418305105031D8A
:100BD000871206305105031D871618305205031D74
:100BE000071206305205031D071618305305031D62
:0C0BF000871106305305031D871508000F
:084000000300030007000100AA
:02400E00CC33B1
:10420000010003000300030003000200020002009B
:104210000200000000000000000003000300030093
:10422000410000000000000000000000000000004D
:104230000000C000C000C000C000C000C000C0003E
:10424000FF00C300F300CF00FF00C300F300CF0066
:10425000FF00C300F300CF00FF00C300F300CF0056
:104260000000FF00FF00FF00FF00FF00FF00FF0055
:10427000FF00FF00FF00FF00FF00FF00FF00FF0046
:10428000FF000300FF00FF00FF00FF00FF00FF0032
:10429000FF00FF00FF00FF00FF00FF00FF00FF0026
:1042A000FF00C000FF00FF00FF00FF00FF00FF0055
:1042B000FF00FF00FF00FF00FF00FF00FF00FF0006
:1042C000FF00FF00FF00FF00FF00FF00FF00FF00F6
:1042D000FF00FF00FF00FF00FF00FF00FF00FF00E6
:1042E000FF00FF00FF00FF00FF00FF00FF00FF00D6
:1042F000FF00FF00FF00FF00FF00FF00FF00AA001B
:00000001FF
